******************************************************************************
               TMS320C6x Linker PC v7.4.2                      
******************************************************************************
>> Linked Fri Jan 03 18:02:38 2014

OUTPUT FILE NAME:   <Multicore_Navigator.out>
ENTRY POINT SYMBOL: "_c_int00"  address: 0c073240


MEMORY CONFIGURATION

         name            origin    length      used     unused   attr    fill
----------------------  --------  ---------  --------  --------  ----  --------
  VECTORS               00800000   00000200  00000200  00000000  RWIX
  LL2_RW_DATA           00800200   0003fe00  0003d510  000028f0  RWIX
  SL2                   0c000000   00100000  00082fc4  0007d03c  RWIX
  DDR3_CODE             80000000   01000000  00000000  01000000  RWIX
  DDR3_R_DATA           81000000   01000000  00000000  01000000  RWIX
  DDR3_RW_DATA          82000000   06000000  00000000  06000000  RWIX
  DDR3_NO_ECC           90000000   10000000  04240000  0bdc0000  RWIX


SEGMENT ALLOCATION MAP

run origin  load origin   length   init length attrs members
----------  ----------- ---------- ----------- ----- -------
00800000    00800000    00000200   00000200    r-x
  00800000    00800000    00000200   00000200    r-x vecs
00800200    00800200    00036080   00000000    rw-
  00800200    00800200    0001e000   00000000    rw- PacketData.buffer_LL2
  0081e200    0081e200    00018080   00000000    rw- QMSS_Data.Descriptor_LL2
00836280    00836280    000061e8   000051e8    rw-
  00836280    00836280    000051e8   000051e8    rw- .far
  0083b468    0083b468    00001000   00000000    rw- .stack
0083c468    0083c468    00000884   00000884    rw-
  0083c468    0083c468    00000884   00000884    rw- .fardata
0083ccf0    0083ccf0    00000920   00000000    rw-
  0083ccf0    0083ccf0    00000800   00000000    rw- .sysmem
  0083d4f0    0083d4f0    00000120   00000000    rw- .cio
0083d610    0083d610    00000104   000000e8    rw-
  0083d610    0083d610    000000e8   000000e8    rw- .neardata
  0083d6f8    0083d6f8    0000001c   00000000    rw- .bss
0c000000    0c000000    00060080   00000000    rw-
  0c000000    0c000000    00040000   00000000    rw- PacketData.buffer_SL2
  0c040000    0c040000    00020080   00000000    rw- QMSS_Data.Descriptor_SL2
0c060080    0c060080    000137e0   000137e0    r-x
  0c060080    0c060080    000137e0   000137e0    r-x .text
0c073860    0c073860    0000c500   00000000    rw-
  0c073860    0c073860    0000c500   00000000    rw- QMSS_Data.linkingRAM1
0c07fd60    0c07fd60    00003264   00003264    r--
  0c07fd60    0c07fd60    00002bf4   00002bf4    r-- .const
  0c082954    0c082954    00000670   00000670    r-- .cinit
90000000    90000000    04240000   00000000    rw-
  90000000    90000000    04060000   00000000    rw- QMSS_Data.Descriptor_DDR
  94060000    94060000    001e0000   00000000    rw- PacketData.buffer_DDR


SECTION ALLOCATION MAP

 output                                  attributes/
section   page    origin      length       input sections
--------  ----  ----------  ----------   ----------------
vecs       0    00800000    00000200     
                  00800000    00000200     MNav_vectors.obj (vecs)

PacketData.buffer_LL2 
*          0    00800200    0001e000     UNINITIALIZED
                  00800200    0001e000     MNav_Init.obj (PacketData.buffer_LL2)

QMSS_Data.Descriptor_LL2 
*          0    0081e200    00018080     UNINITIALIZED
                  0081e200    00018080     MNav_Init.obj (QMSS_Data.Descriptor_LL2)

.far       0    00836280    000051e8     
                  00836280    00005010     MNav_Test.obj (.far) [fill = 0]
                  0083b290    00000140     rts6600e_elf.lib : defs.obj (.far) [fill = 0]
                  0083b3d0    0000006c     KeyStone_common.obj (.far) [fill = 0]
                  0083b43c    00000004     --HOLE--
                  0083b440    00000010     KeyStone_DDR_Init.obj (.far:Core_MPAX)
                  0083b450    00000010     KeyStone_common.obj (.far:Core_MPAX)
                  0083b460    00000008     rts6600e_elf.lib : trgdrv.obj (.far) [fill = 0]

.stack     0    0083b468    00001000     UNINITIALIZED
                  0083b468    00000008     rts6600e_elf.lib : boot.obj (.stack)
                  0083b470    00000ff8     --HOLE--

.fardata   0    0083c468    00000884     
                  0083c468    000001e0     rts6600e_elf.lib : defs.obj (.fardata:_ftable)
                  0083c648    000001e0     MNav_Init.obj (.fardata:freeHostQueueCfgTable)
                  0083c828    00000150     MNav_Init.obj (.fardata:flowCfgTable)
                  0083c978    000000a0     rts6600e_elf.lib : lowlev.obj (.fardata:_stream)
                  0083ca18    00000078                      : lowlev.obj (.fardata:_device)
                  0083ca90    00000060     MNav_Init.obj (.fardata:descMemRegionsCfg)
                  0083caf0    00000050     MNav_Test.obj (.fardata)
                  0083cb40    00000050     MNav_Init.obj (.fardata:freeMonoQueueCfgTable)
                  0083cb90    00000040     KeyStone_common.obj (.fardata:gstruMpuAddrRange)
                  0083cbd0    00000024     KeyStone_common.obj (.fardata:gpTimerRegs)
                  0083cbf4    00000004     rts6600e_elf.lib : defs.obj (.fardata)
                  0083cbf8    00000024     KeyStone_common.obj (.fardata:internal_exception_str)
                  0083cc1c    00000004     --HOLE--
                  0083cc20    00000020     KeyStone_common.obj (.fardata:bus_err_stat_str)
                  0083cc40    00000020     KeyStone_common.obj (.fardata:gCIC_EXC_EN_MASK)
                  0083cc60    00000020     KeyStone_common.obj (.fardata:gpMPU_regs)
                  0083cc80    00000018     KeyStone_common.obj (.fardata:Peri_MPU_err_type_str)
                  0083cc98    00000010     KeyStone_common.obj (.fardata:gpEDMA_TC_regs)
                  0083cca8    0000000c     rts6600e_elf.lib : exit.obj (.fardata)
                  0083ccb4    0000000c                      : memory.obj (.fardata)
                  0083ccc0    00000008     KeyStone_common.obj (.fardata:Ns_str)
                  0083ccc8    00000008     KeyStone_Navigator_init_drv.obj (.fardata:gpQM_PDSP_Cmd)
                  0083ccd0    00000008     KeyStone_Navigator_init_drv.obj (.fardata:gpQM_PDSP_CtrlRegs)
                  0083ccd8    00000008     KeyStone_Navigator_init_drv.obj (.fardata:gpQM_PDSP_IRAM)
                  0083cce0    00000008     rts6600e_elf.lib : _lock.obj (.fardata)
                  0083cce8    00000004     KeyStone_common.obj (.fardata:gpEDMA_CC_regs)

.sysmem    0    0083ccf0    00000800     UNINITIALIZED
                  0083ccf0    00000008     rts6600e_elf.lib : memory.obj (.sysmem)
                  0083ccf8    000007f8     --HOLE--

.cio       0    0083d4f0    00000120     UNINITIALIZED
                  0083d4f0    00000120     rts6600e_elf.lib : trgmsg.obj (.cio)

.neardata 
*          0    0083d610    000000e8     
                  0083d610    00000098     KeyStone_common.obj (.neardata)
                  0083d6a8    00000050     KeyStone_Navigator_init_drv.obj (.neardata)

.rodata    0    0083d6f8    00000000     UNINITIALIZED

.bss       0    0083d6f8    0000001c     UNINITIALIZED
                  0083d6f8    00000010     MNav_Init.obj (.bss)
                  0083d708    00000008     MNav_QM_Intc_setup.obj (.bss)
                  0083d710    00000004     MNav_Test.obj (.bss)

PacketData.buffer_SL2 
*          0    0c000000    00040000     UNINITIALIZED
                  0c000000    00040000     MNav_Init.obj (PacketData.buffer_SL2)

QMSS_Data.Descriptor_SL2 
*          0    0c040000    00020080     UNINITIALIZED
                  0c040000    00020080     MNav_Init.obj (QMSS_Data.Descriptor_SL2)

.text      0    0c060080    000137e0     
                  0c060080    00005f00     KeyStone_common.obj (.text)
                  0c065f80    00002a20     KeyStone_DDR_Init.obj (.text)
                  0c0689a0    00001a80     KeyStone_Navigator_init_drv.obj (.text)
                  0c06a420    00000fe0     MNav_Test.obj (.text)
                  0c06b400    000008c0     MNav_Test_main.obj (.text)
                  0c06bcc0    00000600     KeyStone_common.obj (.text:retain)
                  0c06c2c0    000005c0     rts6600e_elf.lib : divd.obj (.text:__c6xabi_divd)
                  0c06c880    000005c0                      : _printfi.obj (.text:_getarg_diouxp)
                  0c06ce40    000005c0     MNav_Test.obj (.text:retain)
                  0c06d400    000004c0     MNav_Init.obj (.text)
                  0c06d8c0    00000460     rts6600e_elf.lib : _printfi.obj (.text:_printfi)
                  0c06dd20    00000460                      : _printfi.obj (.text:_setfield)
                  0c06e180    00000440     KeyStone_common.obj (.text:Core_MPAX)
                  0c06e5c0    000003a0     rts6600e_elf.lib : fputs.obj (.text:fputs)
                  0c06e960    00000320                      : _printfi.obj (.text:_pproc_fge)
                  0c06ec80    000002e0                      : _printfi.obj (.text:_pproc_fwp)
                  0c06ef60    000002a0     MNav_QM_Intc_setup.obj (.text)
                  0c06f200    000002a0     rts6600e_elf.lib : _printfi.obj (.text:fcvt)
                  0c06f4a0    00000280                      : divf.obj (.text:__c6xabi_divf)
                  0c06f720    00000280                      : _printfi.obj (.text:ecvt)
                  0c06f9a0    00000280                      : memory.obj (.text:free)
                  0c06fc20    00000240                      : imath64.obj (.text:__c6xabi_divull)
                  0c06fe60    00000240                      : _printfi.obj (.text:_pconv_e)
                  0c0700a0    00000240                      : _printfi.obj (.text:_pproc_diouxp)
                  0c0702e0    00000220                      : _printfi.obj (.text:_pproc_str)
                  0c070500    00000220                      : fputc.obj (.text:fputc)
                  0c070720    00000200                      : _printfi.obj (.text:_pconv_g)
                  0c070920    00000200                      : setvbuf.obj (.text:setvbuf)
                  0c070b20    000001c0                      : _printfi.obj (.text:_mcpy)
                  0c070ce0    000001a0                      : trgdrv.obj (.text:HOSTrename)
                  0c070e80    000001a0                      : imath40.obj (.text:__c6xabi_divul)
                  0c071020    00000180                      : copy_decompress_rle.obj (.text:__TI_decompress_rle_core)
                  0c0711a0    00000180                      : memory.obj (.text:malloc)
                  0c071320    00000140                      : _printfi.obj (.text:_pproc_fflags)
                  0c071460    00000140                      : lowlev.obj (.text:getdevice)
                  0c0715a0    00000120                      : fclose.obj (.text:_closefile)
                  0c0716c0    00000120                      : _printfi.obj (.text:_ltostr)
                  0c0717e0    00000120                      : fseek.obj (.text:fseek)
                  0c071900    00000100                      : trgdrv.obj (.text:HOSTlseek)
                  0c071a00    00000100                      : autoinit.obj (.text:_auto_init_elf)
                  0c071b00    00000100                      : _io_perm.obj (.text:_wrt_ok)
                  0c071c00    00000100                      : cpy_tbl.obj (.text:copy_in)
                  0c071d00    000000e0                      : trgdrv.obj (.text:HOSTopen)
                  0c071de0    000000e0                      : _printfi.obj (.text:_div)
                  0c071ec0    000000e0                      : atoi.obj (.text:atoi)
                  0c071fa0    000000e0                      : lowlev.obj (.text:close)
                  0c072080    000000e0                      : copy_zero_init.obj (.text:decompress:ZI:__TI_zero_init)
                  0c072160    000000e0                      : ltoa.obj (.text:ltoa)
                  0c072240    000000e0                      : memset.obj (.text:memset)
                  0c072320    000000e0                      : printf.obj (.text:printf)
                  0c072400    000000c0                      : trgdrv.obj (.text:HOSTread)
                  0c0724c0    000000c0                      : trgdrv.obj (.text:HOSTunlink)
                  0c072580    000000c0                      : trgdrv.obj (.text:HOSTwrite)
                  0c072640    000000c0                      : divu.obj (.text:__divu)
                  0c072700    000000c0                      : fflush.obj (.text:_doflush)
                  0c0727c0    000000c0                      : exit.obj (.text:exit)
                  0c072880    000000c0                      : tls.obj (.text:tls:init:__TI_tls_init)
                  0c072940    000000a0                      : trgdrv.obj (.text:HOSTclose)
                  0c0729e0    000000a0                      : fopen.obj (.text:_cleanup)
                  0c072a80    000000a0                      : _printfi.obj (.text:_ecpy)
                  0c072b20    000000a0                      : _printfi.obj (.text:_fcpy)
                  0c072bc0    000000a0                      : memory.obj (.text:_minit)
                  0c072c60    000000a0                      : _printfi.obj (.text:_pconv_f)
                  0c072d00    000000a0                      : lowlev.obj (.text:finddevice)
                  0c072da0    000000a0                      : lowlev.obj (.text:lseek)
                  0c072e40    000000a0                      : memcpy64.obj (.text:memcpy)
                  0c072ee0    000000a0                      : memory.obj (.text:minsert)
                  0c072f80    000000a0                      : memory.obj (.text:mremove)
                  0c073020    000000a0                      : lowlev.obj (.text:write)
                  0c0730c0    00000080                      : fixdu.obj (.text:__c6xabi_fixdu)
                  0c073140    00000080                      : fixfu.obj (.text:__c6xabi_fixfu)
                  0c0731c0    00000080                      : llshift.obj (.text:__c6xabi_llshl)
                  0c073240    00000080                      : boot.obj (.text:_c_int00)
                  0c0732c0    00000080                      : trgmsg.obj (.text:readmsg)
                  0c073340    00000080                      : lowlev.obj (.text:unlink)
                  0c0733c0    00000060                      : cpp_init.obj (.text:__TI_cpp_init)
                  0c073420    00000060                      : frcmpyd_div.obj (.text:__c6xabi_frcmpyd_div)
                  0c073480    00000060                      : llshift.obj (.text:__c6xabi_llshru)
                  0c0734e0    00000060                      : imath64.obj (.text:_subcull)
                  0c073540    00000060                      : memccpy.obj (.text:memccpy)
                  0c0735a0    00000060                      : trgmsg.obj (.text:writemsg)
                  0c073600    00000040     MNav_vectors.obj (.text)
                  0c073640    00000040     rts6600e_elf.lib : isinf.obj (.text:__c6xabi_isinf)
                  0c073680    00000040                      : _printfi.obj (.text:__c6xabi_isnan)
                  0c0736c0    00000040                      : strasg.obj (.text:__strasgi_64plus)
                  0c073700    00000040                      : args_main.obj (.text:_args_main)
                  0c073740    00000040                      : fputs.obj (.text:puts)
                  0c073780    00000020                      : negll.obj (.text:__c6xabi_negll)
                  0c0737a0    00000020                      : _lock.obj (.text:_nop)
                  0c0737c0    00000020                      : printf.obj (.text:_outc)
                  0c0737e0    00000020                      : printf.obj (.text:_outs)
                  0c073800    00000020                      : exit.obj (.text:abort)
                  0c073820    00000020                      : copy_decompress_none.obj (.text:decompress:none:__TI_decompress_none)
                  0c073840    00000020                      : copy_decompress_rle.obj (.text:decompress:rle24:__TI_decompress_rle24)

QMSS_Data.linkingRAM1 
*          0    0c073860    0000c500     UNINITIALIZED
                  0c073860    0000c500     MNav_Init.obj (QMSS_Data.linkingRAM1)

.const     0    0c07fd60    00002bf4     
                  0c07fd60    00001a34     KeyStone_common.obj (.const:.string)
                  0c081794    00000002     rts6600e_elf.lib : fputs.obj (.const:.string)
                  0c081796    00000002     --HOLE-- [fill = 0]
                  0c081798    00000630     MNav_Init.obj (.const:acc48_be)
                  0c081dc8    00000414     MNav_Test.obj (.const:.string)
                  0c0821dc    000003bc     MNav_Test_main.obj (.const:.string)
                  0c082598    00000154     KeyStone_Navigator_init_drv.obj (.const:.string)
                  0c0826ec    00000004     --HOLE-- [fill = 0]
                  0c0826f0    00000101     rts6600e_elf.lib : ctype.obj (.const:.string:_ctypes_)
                  0c0827f1    00000003     --HOLE-- [fill = 0]
                  0c0827f4    0000008c     MNav_Init.obj (.const:.string)
                  0c082880    0000005c     KeyStone_DDR_Init.obj (.const:.string)
                  0c0828dc    00000004     --HOLE-- [fill = 0]
                  0c0828e0    00000038     KeyStone_common.obj (.const:$P$T0$1)
                  0c082918    00000023     rts6600e_elf.lib : _printfi.obj (.const:.string)
                  0c08293b    00000001     --HOLE-- [fill = 0]
                  0c08293c    00000018     MNav_QM_Intc_setup.obj (.const:.string)

.cinit     0    0c082954    00000670     
                  0c082954    000004b4     (.cinit..fardata.load) [load image, compression = rle]
                  0c082e08    000000eb     (.cinit..neardata.load) [load image, compression = rle]
                  0c082ef3    00000001     --HOLE-- [fill = 0]
                  0c082ef4    0000002a     (.cinit..far.load) [load image, compression = rle]
                  0c082f1e    00000002     --HOLE-- [fill = 0]
                  0c082f20    0000000c     (__TI_handler_table)
                  0c082f2c    00000008     (.cinit..bss.load) [load image, compression = zero_init]
                  0c082f34    00000008     (.cinit.PacketData.buffer_DDR.load) [load image, compression = zero_init]
                  0c082f3c    00000008     (.cinit.PacketData.buffer_LL2.load) [load image, compression = zero_init]
                  0c082f44    00000008     (.cinit.PacketData.buffer_SL2.load) [load image, compression = zero_init]
                  0c082f4c    00000008     (.cinit.QMSS_Data.Descriptor_DDR.load) [load image, compression = zero_init]
                  0c082f54    00000008     (.cinit.QMSS_Data.Descriptor_LL2.load) [load image, compression = zero_init]
                  0c082f5c    00000008     (.cinit.QMSS_Data.Descriptor_SL2.load) [load image, compression = zero_init]
                  0c082f64    00000008     (.cinit.QMSS_Data.linkingRAM1.load) [load image, compression = zero_init]
                  0c082f6c    00000058     (__TI_cinit_table)

QMSS_Data.Descriptor_DDR 
*          0    90000000    04060000     UNINITIALIZED
                  90000000    04060000     MNav_Init.obj (QMSS_Data.Descriptor_DDR)

PacketData.buffer_DDR 
*          0    94060000    001e0000     UNINITIALIZED
                  94060000    001e0000     MNav_Init.obj (PacketData.buffer_DDR)


LINKER GENERATED COPY TABLES

__TI_cinit_table @ 0c082f6c records: 11, size/record: 8, table size: 88
	.fardata: load addr=0c082954, load size=000004b4 bytes, run addr=0083c468, run size=00000884 bytes, compression=rle
	.neardata: load addr=0c082e08, load size=000000eb bytes, run addr=0083d610, run size=000000e8 bytes, compression=rle
	.far: load addr=0c082ef4, load size=0000002a bytes, run addr=00836280, run size=000051e8 bytes, compression=rle
	.bss: load addr=0c082f2c, load size=00000008 bytes, run addr=0083d6f8, run size=0000001c bytes, compression=zero_init
	PacketData.buffer_DDR: load addr=0c082f34, load size=00000008 bytes, run addr=94060000, run size=001e0000 bytes, compression=zero_init
	PacketData.buffer_LL2: load addr=0c082f3c, load size=00000008 bytes, run addr=00800200, run size=0001e000 bytes, compression=zero_init
	PacketData.buffer_SL2: load addr=0c082f44, load size=00000008 bytes, run addr=0c000000, run size=00040000 bytes, compression=zero_init
	QMSS_Data.Descriptor_DDR: load addr=0c082f4c, load size=00000008 bytes, run addr=90000000, run size=04060000 bytes, compression=zero_init
	QMSS_Data.Descriptor_LL2: load addr=0c082f54, load size=00000008 bytes, run addr=0081e200, run size=00018080 bytes, compression=zero_init
	QMSS_Data.Descriptor_SL2: load addr=0c082f5c, load size=00000008 bytes, run addr=0c040000, run size=00020080 bytes, compression=zero_init
	QMSS_Data.linkingRAM1: load addr=0c082f64, load size=00000008 bytes, run addr=0c073860, run size=0000c500 bytes, compression=zero_init


LINKER GENERATED HANDLER TABLE

__TI_handler_table @ 0c082f20 records: 3, size/record: 4, table size: 12
	index: 0, handler: __TI_decompress_rle24
	index: 1, handler: __TI_decompress_none
	index: 2, handler: __TI_zero_init


GLOBAL SYMBOLS: SORTED ALPHABETICALLY BY Name 

address    name
--------   ----
0c0647f0   Bus_error_handler
0c073800   C$$EXIT
0c0735f8   C$$IO$$
0c067ae0   C6657_EVM_DDR_Init
0c06746c   C6670_EVM_DDR_Init
0c0665b0   C6678_EVM_DDR_Init
0c06f084   CIC_Init_QM
0c06608c   DDR3_registers_adress_map
0083b440   DDR_REGS_MPAX_cfg_table
0c06b798   DSPCoreAccessQueueTest
0c066c48   Dual_Nyquist_EVM_DDR_Init
0c062254   EDMA_CC_error_handler
0c062468   EDMA_TC_error_handler
0c06189c   EDMA_TC_priority_cfg
0c061838   EDMA_channel_TC_cfg
0c061c08   EDMA_copy
0c062594   EDMA_error_handler
0c061e14   EDMA_fill
0c0618f0   EDMA_init
0c061b48   EDMA_wait
0c065318   EXC_NMI
0c065258   EXC_internal
0c065330   EXC_swgen
0c06bcc0   Exception_service_routine
0c062fcc   Gauss_MPU4_constant
0c072940   HOSTclose
0c071900   HOSTlseek
0c071d00   HOSTopen
0c072400   HOSTread
0c070ce0   HOSTrename
0c0724c0   HOSTunlink
0c072580   HOSTwrite
0c0621b4   IDMA_copy
0c062188   IDMA_wait
0c0648cc   KeyStone_CIC_EXC_handler
0c0640ec   KeyStone_CIC_exception_events_mapping
0c069434   KeyStone_Copy_FDQ
0c062a44   KeyStone_CorePac_AID_map
0c066294   KeyStone_DDR_ECC_INT_enable
0c0662b8   KeyStone_DDR_ECC_init
0c0611b0   KeyStone_DDR_PLL_init
0c0664a4   KeyStone_DDR_clock_phase_init
0c066100   KeyStone_DDR_full_leveling
0c0687e8   KeyStone_DDR_init
0c066564   KeyStone_DDR_latch_leveling_configuration
0c066190   KeyStone_DDR_read_incremental_leveling
0c064d98   KeyStone_EXC_external
0c0645e4   KeyStone_Exception_cfg
0c069024   KeyStone_Host_Descriptor_Queues_init
0c06e310   KeyStone_MPAX_seg_setup
0c0632a0   KeyStone_MPU_MPPA_modify
0c0633a4   KeyStone_MPU_interrupts_enable
0c06300c   KeyStone_MPU_range_setup
0c06308c   KeyStone_MPU_setup
0c062d08   KeyStone_MSMC_MP_interrupt_en
0c062e88   KeyStone_MSMC_protection_exception_handler
0c0692a0   KeyStone_Mono_Descriptor_Queues_init
0c061018   KeyStone_PLL_init
0c062acc   KeyStone_PrivID_Remap
0c068c38   KeyStone_QMSS_Descriptor_Regions_init
0c068b68   KeyStone_QMSS_Linking_RAM_init
0c0696c0   KeyStone_Qmss_Config_Acc_Channel
0c0699f0   KeyStone_Qmss_Config_Reclaim_Queue
0c069500   KeyStone_Qmss_Download_Firmware
0c069984   KeyStone_Qmss_config_Acc_Timer
0c0698b8   KeyStone_Qmss_disable_Acc_Channel
0c062c28   KeyStone_SES_MPAX_setup
0c0637d4   KeyStone_SL2_EDC_enable
0c063e08   KeyStone_SL2_EDC_handler
0c063894   KeyStone_SL2_EDC_interrupt_en
0c062b48   KeyStone_SMS_MPAX_setup
0c06e4b4   KeyStone_XMC_MPAX_setup
0c0617ec   KeyStone_disable_PSC_Power_Domain
0c061794   KeyStone_disable_PSC_module
0c061730   KeyStone_enable_PSC_module
0c060b8c   KeyStone_main_PLL_init
0c0636ec   KeyStone_peripherals_MPU_excepiton_handler
0c0635ec   KeyStone_peripherals_MPU_fault_status
0c069a58   KeyStone_pktDma_Global_Control
0c069ac0   KeyStone_pktDma_TxCh_config
0c069b18   KeyStone_pktDma_configureRxFlow
0c065348   KeyStone_print_device_info
0c062770   L1D_memory_protection_cfg
0c063a50   L1P_EDC_setup
0c063ce4   L1P_ED_handler
0c0626e0   L1P_memory_protection_cfg
0c062638   L1_MPPA_setup
0c062804   L1_cache_protection
0083d694   LL2_EDC_DMA_err_str
0083d698   LL2_EDC_L1D_err_str
0083d69c   LL2_EDC_L1P_err_str
0c063ad4   LL2_EDC_handler
0c0639b4   LL2_EDC_scrub
0c0638ec   LL2_EDC_setup
0083d690   LL2_EDC_victim_err_str
0c062814   LL2_MPPA_setup
0c0628b0   LL2_Memory_Protection_cfg
0c065a8c   Memory_Address_Bus_Test
0c0653e0   Memory_Address_Test
0c065660   Memory_Data_Bus_Test
0c065524   Memory_Fill_Test
0c065ef0   Memory_quick_test
0c06c070   Nested_Exception_service_routine
0083ccc0   Ns_str
0083cc80   Peri_MPU_err_type_str
0c06b870   PktDmaTest
0c06af78   PktDmaThroughput
0c06b818   PktDmaThroughputTest
0c06d4f8   QMSS_PktDMA_init
0c06d440   QMSS_init
0c06f14c   QM_Interrupts_Init
0c06ce40   QueueAccumulationISR
0c06d1e0   QueuePendISR
0c06b7cc   QueuePendInterruptTest
0c06a944   QueuePopCycleTest
0c06a7d8   QueuePushCycleTest
0c06b560   QueuePushPopTest
0c06ab50   QueuePushToAccumulationDelayTest
0c06ae2c   QueuePushToPendInterruptDelayTest
0c06aa78   QueuePushToPopDelayTest
0c06ae94   QueueReclamationDelayTest
0c0613ec   Reset_Timer
0c06d56c   SRIO_PktDMA_init
0c0616ec   Service_Watchdog
0c068118   TCI6614_EVM_DDR_Init
0c062f80   TN_MPU5_constant
0c0612a8   TSC_delay_ms
0c061348   TSC_delay_us
0c061294   TSC_init
0c061440   Timer64_Init
0083d4f0   __CIOBUF_
0c082f6c   __TI_CINIT_Base
0c082fc4   __TI_CINIT_Limit
0c082f20   __TI_Handler_Table_Base
0c082f2c   __TI_Handler_Table_Limit
UNDEFED    __TI_INITARRAY_Base
UNDEFED    __TI_INITARRAY_Limit
0083c468   __TI_STACK_END
00001000   __TI_STACK_SIZE
0083d610   __TI_STATIC_BASE
00000800   __TI_SYSMEM_SIZE
UNDEFED    __TI_TLS_INIT_Base
UNDEFED    __TI_TLS_INIT_Limit
00000001   __TI_args_main
0c0733c0   __TI_cpp_init
0c073820   __TI_decompress_none
0c073840   __TI_decompress_rle24
0083ccb0   __TI_enable_exit_profile_output
ffffffff   __TI_pprof_out_hndl
ffffffff   __TI_prof_data_size
ffffffff   __TI_prof_data_start
0c072880   __TI_tls_init
0c072080   __TI_zero_init
ffffffff   __binit__
0c06c2c0   __c6xabi_divd
0c06f4a0   __c6xabi_divf
0c072640   __c6xabi_divu
0c070e80   __c6xabi_divul
0c06fc20   __c6xabi_divull
0c0730c0   __c6xabi_fixdu
0c073140   __c6xabi_fixfu
0c073420   __c6xabi_frcmpyd_div
0c073640   __c6xabi_isinf
0c0731c0   __c6xabi_llshl
0c073480   __c6xabi_llshru
0c073780   __c6xabi_negll
0c0736c0   __c6xabi_strasgi_64plus
ffffffff   __c_args__
0c072640   __divu
0c0736c0   __strasgi_64plus
0c073700   _args_main
0c071a00   _auto_init_elf
0c073240   _c_int00
0c0729e0   _cleanup
0083cca8   _cleanup_ptr
0c0715a0   _closefile
0c0826f0   _ctypes_
0c072700   _doflush
0083ccac   _dtors_ptr
0083cbf4   _ft_end
0083c468   _ftable
0083cce0   _lock
0c072bc0   _minit
0c0737a0   _nop
0c06d8c0   _printfi
0083b468   _stack
0c0734e0   _subcull
0083ccf0   _sys_memory
0083b290   _tmpnams
0083cce4   _unlock
0c071b00   _wrt_ok
0c073800   abort
0c081798   acc48_be
0c071ec0   atoi
ffffffff   binit
0083cc20   bus_err_stat_str
0c061240   calc_cycle_measure_overhead
0c06d5d0   checkQueues
0c071fa0   close
0c071c00   copy_in
0083d688   cycle_measure_overhead
0083ca90   descMemRegionsCfg
0083b3d0   exception_record
0c0727c0   exit
0083c828   flowCfgTable
0c070500   fputc
0c06e5c0   fputs
0c06f9a0   free
0083c648   freeHostQueueCfgTable
0083cb40   freeMonoQueueCfgTable
0c0717e0   fseek
0083cc40   gCIC_EXC_EN_MASK
0083d6a4   gCIC_EXC_out_num
0083d684   gDSP_Core_Speed_Hz
0083d618   gpBootCfgRegs
0083d614   gpCGEM_regs
0083d62c   gpCIC0_regs
0083d630   gpCIC1_regs
0083d634   gpCIC_regs
0083d680   gpDDR_regs
0083d638   gpEDMA_CC2_regs
0083cce8   gpEDMA_CC_regs
0083d63c   gpEDMA_TC_2_0_regs
0083d640   gpEDMA_TC_2_1_regs
0083d644   gpEDMA_TC_2_2_regs
0083d648   gpEDMA_TC_2_3_regs
0083cc98   gpEDMA_TC_regs
0083d628   gpGPIO_regs
0083d670   gpMPU0_regs
0083d674   gpMPU1_regs
0083d678   gpMPU2_regs
0083d67c   gpMPU3_regs
0083cc60   gpMPU_regs
0083d624   gpMSMC_regs
0083d61c   gpPLLC_regs
0083d620   gpPSC_regs
0083d6cc   gpQM_DMA_CfgRegs
0083d6d4   gpQM_DMA_RxChCfgRegs
0083d6dc   gpQM_DMA_RxFlowCfgRegs
0083d6d0   gpQM_DMA_TxChCfgRegs
0083d6d8   gpQM_DMA_TxChPriority
0083d6c8   gpQM_INTD_regs
0083ccc8   gpQM_PDSP_Cmd
0083ccd0   gpQM_PDSP_CtrlRegs
0083ccd8   gpQM_PDSP_IRAM
0083d6a8   gpQM_configRegs
0083d6ac   gpQM_descriptorRegions
0083d6b4   gpQueueManageProxyRegs
0083d6bc   gpQueueManageProxyVBUSM
0083d6b0   gpQueueManageRegs
0083d6b8   gpQueueManageVBUSM
0083d6c0   gpQueueStatusConfigRegs
0083d6c4   gpQueueThresholdStatus
0083d6e0   gpSRIO_DMA_CfgRegs
0083d6e8   gpSRIO_DMA_RxChCfgRegs
0083d6f0   gpSRIO_DMA_RxFlowCfgRegs
0083d6e4   gpSRIO_DMA_TxChCfgRegs
0083d6ec   gpSRIO_DMA_TxChPriority
0083d64c   gpTimer0Regs
0083d650   gpTimer1Regs
0083d654   gpTimer2Regs
0083d658   gpTimer3Regs
0083d65c   gpTimer4Regs
0083d660   gpTimer5Regs
0083d664   gpTimer6Regs
0083d668   gpTimer7Regs
0083d66c   gpTimer8Regs
0083cbd0   gpTimerRegs
0083d610   gpXMC_regs
0083cb90   gstruMpuAddrRange
0083d6a0   guwIntcCICExcEvtIdx
0083caf0   hiQuAccCfg
90000000   hostDescriptor_DDR
0081e200   hostDescriptor_LL2
0c040000   hostDescriptor_SL2
0083d710   intTSCL
0083cbf8   internal_exception_str
0c073860   linkingRAM1
0083cb18   loQuAccCfg
0c06e180   lock_mem_prot_regs
0c072da0   lseek
0c072160   ltoa
0c06ba00   main
0c0711a0   malloc
0083b450   mem_prot_key
0c073540   memccpy
0c072e40   memcpy
0c062d70   memory_protection_exception_handler
0c072240   memset
90040000   monoDescriptor_DDR
00826200   monoDescriptor_LL2
0c050000   monoDescriptor_SL2
0083d6f4   numLinkingEntry
94060000   packetBuffer_DDR_Size0
94080000   packetBuffer_DDR_Size1
940c0000   packetBuffer_DDR_Size2
94140000   packetBuffer_DDR_Size3
00800200   packetBuffer_LL2_Size0
00802200   packetBuffer_LL2_Size1
00806200   packetBuffer_LL2_Size2
0080e200   packetBuffer_LL2_Size3
0c000000   packetBuffer_SL2_Size0
0c010000   packetBuffer_SL2_Size1
0c020000   packetBuffer_SL2_Size2
0c030000   packetBuffer_SL2_Size3
0c072320   printf
0c073740   puts
0c0732c0   readmsg
0c073340   remove
0c070920   setvbuf
0083d6fc   uiInitialHostFdqNum
0083d700   uiInitialMonoFdqNum
0083d68c   uiLL2_scrub_addr
0083d70c   uiQ662_pend_host_event_num
0083d708   uiQ662_pend_system_event_num
0083d6f8   uiUsedDescRegionNum
0083d704   uiUsedRxFlowNum
00836280   uiaDescriptorBuffer
00837280   uiaDescriptorPingPongBufferHi
00839288   uiaDescriptorPingPongBufferLo
0c073340   unlink
0c06e248   unlock_mem_prot_regs
00800000   vectors
0c073020   write
0c0735a0   writemsg


GLOBAL SYMBOLS: SORTED BY Symbol Address 

address    name
--------   ----
00000001   __TI_args_main
00000800   __TI_SYSMEM_SIZE
00001000   __TI_STACK_SIZE
00800000   vectors
00800200   packetBuffer_LL2_Size0
00802200   packetBuffer_LL2_Size1
00806200   packetBuffer_LL2_Size2
0080e200   packetBuffer_LL2_Size3
0081e200   hostDescriptor_LL2
00826200   monoDescriptor_LL2
00836280   uiaDescriptorBuffer
00837280   uiaDescriptorPingPongBufferHi
00839288   uiaDescriptorPingPongBufferLo
0083b290   _tmpnams
0083b3d0   exception_record
0083b440   DDR_REGS_MPAX_cfg_table
0083b450   mem_prot_key
0083b468   _stack
0083c468   __TI_STACK_END
0083c468   _ftable
0083c648   freeHostQueueCfgTable
0083c828   flowCfgTable
0083ca90   descMemRegionsCfg
0083caf0   hiQuAccCfg
0083cb18   loQuAccCfg
0083cb40   freeMonoQueueCfgTable
0083cb90   gstruMpuAddrRange
0083cbd0   gpTimerRegs
0083cbf4   _ft_end
0083cbf8   internal_exception_str
0083cc20   bus_err_stat_str
0083cc40   gCIC_EXC_EN_MASK
0083cc60   gpMPU_regs
0083cc80   Peri_MPU_err_type_str
0083cc98   gpEDMA_TC_regs
0083cca8   _cleanup_ptr
0083ccac   _dtors_ptr
0083ccb0   __TI_enable_exit_profile_output
0083ccc0   Ns_str
0083ccc8   gpQM_PDSP_Cmd
0083ccd0   gpQM_PDSP_CtrlRegs
0083ccd8   gpQM_PDSP_IRAM
0083cce0   _lock
0083cce4   _unlock
0083cce8   gpEDMA_CC_regs
0083ccf0   _sys_memory
0083d4f0   __CIOBUF_
0083d610   __TI_STATIC_BASE
0083d610   gpXMC_regs
0083d614   gpCGEM_regs
0083d618   gpBootCfgRegs
0083d61c   gpPLLC_regs
0083d620   gpPSC_regs
0083d624   gpMSMC_regs
0083d628   gpGPIO_regs
0083d62c   gpCIC0_regs
0083d630   gpCIC1_regs
0083d634   gpCIC_regs
0083d638   gpEDMA_CC2_regs
0083d63c   gpEDMA_TC_2_0_regs
0083d640   gpEDMA_TC_2_1_regs
0083d644   gpEDMA_TC_2_2_regs
0083d648   gpEDMA_TC_2_3_regs
0083d64c   gpTimer0Regs
0083d650   gpTimer1Regs
0083d654   gpTimer2Regs
0083d658   gpTimer3Regs
0083d65c   gpTimer4Regs
0083d660   gpTimer5Regs
0083d664   gpTimer6Regs
0083d668   gpTimer7Regs
0083d66c   gpTimer8Regs
0083d670   gpMPU0_regs
0083d674   gpMPU1_regs
0083d678   gpMPU2_regs
0083d67c   gpMPU3_regs
0083d680   gpDDR_regs
0083d684   gDSP_Core_Speed_Hz
0083d688   cycle_measure_overhead
0083d68c   uiLL2_scrub_addr
0083d690   LL2_EDC_victim_err_str
0083d694   LL2_EDC_DMA_err_str
0083d698   LL2_EDC_L1D_err_str
0083d69c   LL2_EDC_L1P_err_str
0083d6a0   guwIntcCICExcEvtIdx
0083d6a4   gCIC_EXC_out_num
0083d6a8   gpQM_configRegs
0083d6ac   gpQM_descriptorRegions
0083d6b0   gpQueueManageRegs
0083d6b4   gpQueueManageProxyRegs
0083d6b8   gpQueueManageVBUSM
0083d6bc   gpQueueManageProxyVBUSM
0083d6c0   gpQueueStatusConfigRegs
0083d6c4   gpQueueThresholdStatus
0083d6c8   gpQM_INTD_regs
0083d6cc   gpQM_DMA_CfgRegs
0083d6d0   gpQM_DMA_TxChCfgRegs
0083d6d4   gpQM_DMA_RxChCfgRegs
0083d6d8   gpQM_DMA_TxChPriority
0083d6dc   gpQM_DMA_RxFlowCfgRegs
0083d6e0   gpSRIO_DMA_CfgRegs
0083d6e4   gpSRIO_DMA_TxChCfgRegs
0083d6e8   gpSRIO_DMA_RxChCfgRegs
0083d6ec   gpSRIO_DMA_TxChPriority
0083d6f0   gpSRIO_DMA_RxFlowCfgRegs
0083d6f4   numLinkingEntry
0083d6f8   uiUsedDescRegionNum
0083d6fc   uiInitialHostFdqNum
0083d700   uiInitialMonoFdqNum
0083d704   uiUsedRxFlowNum
0083d708   uiQ662_pend_system_event_num
0083d70c   uiQ662_pend_host_event_num
0083d710   intTSCL
0c000000   packetBuffer_SL2_Size0
0c010000   packetBuffer_SL2_Size1
0c020000   packetBuffer_SL2_Size2
0c030000   packetBuffer_SL2_Size3
0c040000   hostDescriptor_SL2
0c050000   monoDescriptor_SL2
0c060b8c   KeyStone_main_PLL_init
0c061018   KeyStone_PLL_init
0c0611b0   KeyStone_DDR_PLL_init
0c061240   calc_cycle_measure_overhead
0c061294   TSC_init
0c0612a8   TSC_delay_ms
0c061348   TSC_delay_us
0c0613ec   Reset_Timer
0c061440   Timer64_Init
0c0616ec   Service_Watchdog
0c061730   KeyStone_enable_PSC_module
0c061794   KeyStone_disable_PSC_module
0c0617ec   KeyStone_disable_PSC_Power_Domain
0c061838   EDMA_channel_TC_cfg
0c06189c   EDMA_TC_priority_cfg
0c0618f0   EDMA_init
0c061b48   EDMA_wait
0c061c08   EDMA_copy
0c061e14   EDMA_fill
0c062188   IDMA_wait
0c0621b4   IDMA_copy
0c062254   EDMA_CC_error_handler
0c062468   EDMA_TC_error_handler
0c062594   EDMA_error_handler
0c062638   L1_MPPA_setup
0c0626e0   L1P_memory_protection_cfg
0c062770   L1D_memory_protection_cfg
0c062804   L1_cache_protection
0c062814   LL2_MPPA_setup
0c0628b0   LL2_Memory_Protection_cfg
0c062a44   KeyStone_CorePac_AID_map
0c062acc   KeyStone_PrivID_Remap
0c062b48   KeyStone_SMS_MPAX_setup
0c062c28   KeyStone_SES_MPAX_setup
0c062d08   KeyStone_MSMC_MP_interrupt_en
0c062d70   memory_protection_exception_handler
0c062e88   KeyStone_MSMC_protection_exception_handler
0c062f80   TN_MPU5_constant
0c062fcc   Gauss_MPU4_constant
0c06300c   KeyStone_MPU_range_setup
0c06308c   KeyStone_MPU_setup
0c0632a0   KeyStone_MPU_MPPA_modify
0c0633a4   KeyStone_MPU_interrupts_enable
0c0635ec   KeyStone_peripherals_MPU_fault_status
0c0636ec   KeyStone_peripherals_MPU_excepiton_handler
0c0637d4   KeyStone_SL2_EDC_enable
0c063894   KeyStone_SL2_EDC_interrupt_en
0c0638ec   LL2_EDC_setup
0c0639b4   LL2_EDC_scrub
0c063a50   L1P_EDC_setup
0c063ad4   LL2_EDC_handler
0c063ce4   L1P_ED_handler
0c063e08   KeyStone_SL2_EDC_handler
0c0640ec   KeyStone_CIC_exception_events_mapping
0c0645e4   KeyStone_Exception_cfg
0c0647f0   Bus_error_handler
0c0648cc   KeyStone_CIC_EXC_handler
0c064d98   KeyStone_EXC_external
0c065258   EXC_internal
0c065318   EXC_NMI
0c065330   EXC_swgen
0c065348   KeyStone_print_device_info
0c0653e0   Memory_Address_Test
0c065524   Memory_Fill_Test
0c065660   Memory_Data_Bus_Test
0c065a8c   Memory_Address_Bus_Test
0c065ef0   Memory_quick_test
0c06608c   DDR3_registers_adress_map
0c066100   KeyStone_DDR_full_leveling
0c066190   KeyStone_DDR_read_incremental_leveling
0c066294   KeyStone_DDR_ECC_INT_enable
0c0662b8   KeyStone_DDR_ECC_init
0c0664a4   KeyStone_DDR_clock_phase_init
0c066564   KeyStone_DDR_latch_leveling_configuration
0c0665b0   C6678_EVM_DDR_Init
0c066c48   Dual_Nyquist_EVM_DDR_Init
0c06746c   C6670_EVM_DDR_Init
0c067ae0   C6657_EVM_DDR_Init
0c068118   TCI6614_EVM_DDR_Init
0c0687e8   KeyStone_DDR_init
0c068b68   KeyStone_QMSS_Linking_RAM_init
0c068c38   KeyStone_QMSS_Descriptor_Regions_init
0c069024   KeyStone_Host_Descriptor_Queues_init
0c0692a0   KeyStone_Mono_Descriptor_Queues_init
0c069434   KeyStone_Copy_FDQ
0c069500   KeyStone_Qmss_Download_Firmware
0c0696c0   KeyStone_Qmss_Config_Acc_Channel
0c0698b8   KeyStone_Qmss_disable_Acc_Channel
0c069984   KeyStone_Qmss_config_Acc_Timer
0c0699f0   KeyStone_Qmss_Config_Reclaim_Queue
0c069a58   KeyStone_pktDma_Global_Control
0c069ac0   KeyStone_pktDma_TxCh_config
0c069b18   KeyStone_pktDma_configureRxFlow
0c06a7d8   QueuePushCycleTest
0c06a944   QueuePopCycleTest
0c06aa78   QueuePushToPopDelayTest
0c06ab50   QueuePushToAccumulationDelayTest
0c06ae2c   QueuePushToPendInterruptDelayTest
0c06ae94   QueueReclamationDelayTest
0c06af78   PktDmaThroughput
0c06b560   QueuePushPopTest
0c06b798   DSPCoreAccessQueueTest
0c06b7cc   QueuePendInterruptTest
0c06b818   PktDmaThroughputTest
0c06b870   PktDmaTest
0c06ba00   main
0c06bcc0   Exception_service_routine
0c06c070   Nested_Exception_service_routine
0c06c2c0   __c6xabi_divd
0c06ce40   QueueAccumulationISR
0c06d1e0   QueuePendISR
0c06d440   QMSS_init
0c06d4f8   QMSS_PktDMA_init
0c06d56c   SRIO_PktDMA_init
0c06d5d0   checkQueues
0c06d8c0   _printfi
0c06e180   lock_mem_prot_regs
0c06e248   unlock_mem_prot_regs
0c06e310   KeyStone_MPAX_seg_setup
0c06e4b4   KeyStone_XMC_MPAX_setup
0c06e5c0   fputs
0c06f084   CIC_Init_QM
0c06f14c   QM_Interrupts_Init
0c06f4a0   __c6xabi_divf
0c06f9a0   free
0c06fc20   __c6xabi_divull
0c070500   fputc
0c070920   setvbuf
0c070ce0   HOSTrename
0c070e80   __c6xabi_divul
0c0711a0   malloc
0c0715a0   _closefile
0c0717e0   fseek
0c071900   HOSTlseek
0c071a00   _auto_init_elf
0c071b00   _wrt_ok
0c071c00   copy_in
0c071d00   HOSTopen
0c071ec0   atoi
0c071fa0   close
0c072080   __TI_zero_init
0c072160   ltoa
0c072240   memset
0c072320   printf
0c072400   HOSTread
0c0724c0   HOSTunlink
0c072580   HOSTwrite
0c072640   __c6xabi_divu
0c072640   __divu
0c072700   _doflush
0c0727c0   exit
0c072880   __TI_tls_init
0c072940   HOSTclose
0c0729e0   _cleanup
0c072bc0   _minit
0c072da0   lseek
0c072e40   memcpy
0c073020   write
0c0730c0   __c6xabi_fixdu
0c073140   __c6xabi_fixfu
0c0731c0   __c6xabi_llshl
0c073240   _c_int00
0c0732c0   readmsg
0c073340   remove
0c073340   unlink
0c0733c0   __TI_cpp_init
0c073420   __c6xabi_frcmpyd_div
0c073480   __c6xabi_llshru
0c0734e0   _subcull
0c073540   memccpy
0c0735a0   writemsg
0c0735f8   C$$IO$$
0c073640   __c6xabi_isinf
0c0736c0   __c6xabi_strasgi_64plus
0c0736c0   __strasgi_64plus
0c073700   _args_main
0c073740   puts
0c073780   __c6xabi_negll
0c0737a0   _nop
0c073800   C$$EXIT
0c073800   abort
0c073820   __TI_decompress_none
0c073840   __TI_decompress_rle24
0c073860   linkingRAM1
0c081798   acc48_be
0c0826f0   _ctypes_
0c082f20   __TI_Handler_Table_Base
0c082f2c   __TI_Handler_Table_Limit
0c082f6c   __TI_CINIT_Base
0c082fc4   __TI_CINIT_Limit
90000000   hostDescriptor_DDR
90040000   monoDescriptor_DDR
94060000   packetBuffer_DDR_Size0
94080000   packetBuffer_DDR_Size1
940c0000   packetBuffer_DDR_Size2
94140000   packetBuffer_DDR_Size3
ffffffff   __TI_pprof_out_hndl
ffffffff   __TI_prof_data_size
ffffffff   __TI_prof_data_start
ffffffff   __binit__
ffffffff   __c_args__
ffffffff   binit
UNDEFED    __TI_INITARRAY_Base
UNDEFED    __TI_INITARRAY_Limit
UNDEFED    __TI_TLS_INIT_Base
UNDEFED    __TI_TLS_INIT_Limit

[325 symbols]
